:1000000000308A001F29000000000A108A100A111F
:10001000820728340C34013406340A108A100A117D
:100020008207303431343234333434343534363476
:100030003734383439344134423443344434453429
:1000400046340A108A100A1182075234653461342A
:10005000643479342E342E342E34003412080319CB
:100060003E2801308D008C018C0B34288D0B3328F9
:1000700027308C008C0B3A28920B312800340F303B
:10008000860519088C008C0EF0308C050C0886044F
:10009000000086150000861100348610F1306600DD
:1000A00006150000861500000608F0399900861133
:1000B0000000861506089800980E0F3098058611E6
:1000C00001306600190818048D000D089800981B6F
:1000D0004E2886109608031D8614000006110000A5
:1000E000861117089800980E0F3098051808990087
:1000F0003F2017080F399800180899003F20003456
:10010000FF308500E8306500F13086000130660080
:100110008E01643092002E200130900004301002D5
:1001200003189A28033099003F20053092002E20B2
:10013000900A8E28023099003F209001043010026E
:100140000318AB28100805209100960111089700AC
:100150004D20900A9E282329013013020319B32849
:1001600040309400B428940101301202940714081E
:10017000803895009601150897004D20003411082D
:100180008C000C300C020319DA280A300C02031917
:10019000E2280D300C020319E82808300C0203197C
:1001A000EE280E300C020319F3280F300C0203194D
:1001B000F528F7289601013097004D200230920073
:1001C0002E20FD280130920002309300AC20FD2843
:1001D0000130920001309300AC20FD2896011030D0
:1001E00097004D20FD280512FD280516FD28013039
:1001F0009600110897004D20FD28003408308C002F
:100200000618002990018C1713298C131329031049
:10021000900C061890170C1713290C138C0B072938
:1002200010088D001E2919308C1B06308D008D0B97
:1002300017298C1B05290C1B0D290729312984013D
:100240008301061480280C309100BF209001100813
:100250002120003803193029900A9100BF20272956
:10026000FE280D088F00851D39290F089100BF2039
:1002700064290F088C008C0E0F308C050C080D20A3
:10028000900010089100BF200F080F390D2090003A
:1002900010089100BF2020309100BF200E088E0A68
:1002A00005300E02031D5A290130920002309300DE
:1002B000AC2064290A300E02031D64298E0101302E
:0C02C000920001309300AC203029630054
:02400E00F93F78
:084000000D0001000F00050096
:00000001FF
